:030000000219FDE5
:03000B000200AA46
:03002B0002018748
:03005B000203415C
:0300730002032E57
:1000800002030406080C10182030406080040608A3
:100090000C10182030406080A0C00003070F1F0D17
:1000A0000D04050D050305030302C2AF306308C24A
:1000B0006385798AD2AF32C0D0C0E0206221E525C5
:1000C0006016E473E525F4C3334009758A00D263F2
:1000D000F57901D6F58AD262D0E0D0D0D2AF32C362
:1000E000E526334009758A00D263F57901F0F58A77
:1000F000C262E526F4602F30682520720DD0E0D072
:10010000D0C292C294C296D2AF32C292C294C29668
:10011000206F0C206509740AD5E0FDE57B4290D084
:10012000E0D0D0D2AF32758A00D263757900C28D2B
:10013000D262211F01C4306805206502D29201C439
:10014000306805206502D29401C43068052065023C
:10015000D29601C4C29330680A2065077408D5E0BE
:10016000FDD29201C4C29530680A2065077408D593
:10017000E0FDD29401C4C29730680A206507740874
:10018000D5E0FDD29601C4C2AFC2AD53E6EFC0D0F8
:10019000C0E0D2D3D2AFE57A6009E5776005757724
:1001A0000041DB757701C2CEE52A600720744F1548
:1001B0002A21FE7800790020742EE580307E01F43B
:1001C00030E60278FF53DACF207E0343DA20307E18
:1001D0000343DA10C2D8C271E580307E01F430E604
:1001E0000279FFC3E89970CB306103752A18207437
:1001F00003752A18885CD270E86003755F0020746C
:100200000DE52B6004152B410E43DA01C2D8207096
:1002100002417DA85C206102C2702074367982B7E9
:100220000431C3E894F0400374F0F8E8C4540F2894
:10023000F87984B703024153C313C31387212008FD
:1002400002C313200A06C3C898F8415328F8500384
:1002500074FFF88822E52D54066022206B1FE536D6
:10026000C333C333F8E564C313C313F9C395224002
:10027000028922E82522F52250037522FF7882B6F2
:100280000459852224A824C3E52495614002A8616D
:10029000C3E895634002A8638825E566700241CEF5
:1002A000C3E8AA669A5003E8FAE4F9EAC333FBE527
:1002B00068F45B29400D2567F8E567600215674023
:1002C0000B41CE0AC3E5679A5002056778FF88267E
:1002D000C26FC3E52694F84002D26F20CF0AD0E067
:1002E000D0D043E610D2AD32C2CF053AE57A6009EC
:1002F000E578600575780061247578017801E52A54
:100300006005307402152AC3E55C94014005755FF1
:10031000006124756000756900E55F2401F55F5098
:1003200003755FFFD0E0D0D043E610D2AD32C2AF4C
:1003300053E67F7592FA7593FFC260759104D2AF50
:1003400032C2AF53E6EFC2ADC0D0C0E0C0F0D2D3EE
:10035000D2AFA8FBA9FCE57A6007C3E913F9E8135B
:10036000F8C2D830710261B353DACF207E0343DA8A
:1003700010307E0343DA20D271E580307E01F42014
:10038000E602618A88278928A1E053DACF207E031C
:1003900043DA20307E0343DA10C2D8C271307402CF
:1003A000A1CC7800E580307E01F430E602A1CC8853
:1003B0005CA1B453DACF207E0343DA20307E0343BE
:1003C000DA10C271206102818C53DACF207E0343A0
:1003D000DA10307E0343DA20C2D8D27188578958A8
:1003E000C3E89555F8E99556F97B007E087A00C375
:1003F000E8948CE994005005755B00817E88217833
:10040000A2E6A8216055C3E894C8E994005008E426
:10041000D2E4FB7A0A8159C3E89468E99401500850
:10042000E4D2E3FB7A0F8159C3E894D0E9940250F7
:1004300008E4D2E2FB7A1E8159C3E894A0E994054E
:100440005008E4D2E1FB7A3C8159C3E89498E994DE
:10045000085008E4D2E0FB7A787E00C3E89559FCA6
:10046000E9955AFD30E70AECF42401FCEDF4340080
:0E047000FD755B00C3EC9AED9E5003755B01B9
:10047E008859895A8557558558567802A1B4C3E8CC
:10048E009527F8E99528F9307C02A198307B02A1D6
:10049E0098307A02A19120750281AFE9FDE8FC81C6
:1004AE00CEE9C313F9E813F8307902A191E9C31329
:1004BE00F9E813F8307802A191E9C313FDE813FCB3
:1004CE0020612CC3EC941CED9402400281E5ED708A
:1004DE001EC3EC94C850180529E52970021529C3CE
:1004EE00E529940A5002A1CC755C00D270A1CCE52E
:1004FE0029600215297888E6F97400207F0878961D
:10050E00B90302789EE624FAFEE43400FFC3EC9EA3
:10051E00FCED9FFD9208B90310A208500720760942
:10052E00D276A137307602C276A2085016B9030DE4
:10053E00ECF42401FCEDF43400FD02055178007951
:10054E0000A198B90315EC33FCED33FDC3EC940A0E
:10055E00FCED9400FD50047C007D00C3EC94FFED97
:10056E009400400678FF7900A198EC8572F0A4C53E
:10057E00F0A2F733F8790040030205B478FF790052
:10058E000205B4E9C313F9E813F8307C0EE96002F2
:10059E0078FFC3E81338F8E43400F9C3E894FFE9B0
:1005AE009400400278FF885CD270206102A1CC7466
:1005BE001FF4552F4BF52FC274EB7002D274752AAF
:1005CE0018307403752A0A306102A1E020740353B7
:1005DE00DAFE207403752B06D0F0D0E0D0D0D2AD69
:1005EE0043E6103279010206107903020610790AE9
:1005FE00020610791E020610796402061079C802EE
:10060E0006107817E4D5E0FDD8FAD9F6227A147BD5
:10061E00780206377A107B8C0206377A0D7BB4028D
:10062E0006377A0B7BC8020637E573D5E0012279CF
:10063E0002E4C295D5E0FDD294D5E0FDC294D5E09A
:10064E00FDD295D5E0FDE920E002D29230E002D253
:10065E0096E573D5E0FDE920E002C29230E002C2D9
:10066E00967496D5E0FDD9C9EAF8D5E0FDD8FBDB46
:10067E00B8C29522C37C007D0075F00005F0EA3308
:10068E00FAEB33FB50F6EB13FBEA13FAC3E9FFE880
:10069E00FEE89AF8E99BF95004EFF9EEF8B3EC3363
:1006AE00FCED33FDD5F0DFEDF9ECF822E889F08AA8
:1006BE0020D2D4F8A9F07B0030F70B7BFFF4240195
:1006CE00F8E9F43400F9E88520F0A4ADF0F8E985F6
:1006DE0020F0A4AFF0FEED2EF974003FFA7C04C3B7
:1006EE00EA13FAE913F9E813F8DCF48BF030F70AA1
:1006FE00E8F42401F8E9F43400F9E889F0C2D4F8FA
:10070E00A9F0227882B6040302076CC3E55C94015B
:10071E004003020736852224E4F544F545F546F5F7
:10072E0047F548C26E02076C7882E6FCD26EE5226F
:10073E00F523783879C7AA40AB41C3EB13FBEA1314
:10074E00FAEC146013C3EB13FBEA13FAEC14146007
:10075E0007C3EB13FBEA13FAD1828844894522C3FF
:10076E00E5449523F8E5459400F9500CC3E89480D0
:10077E00E994FF401602079DC3E8947FE994005068
:10078E000302079D787F790002079D788079FF88A4
:10079E0049894A22E5492546F8E54A3547F9854A09
:1007AE0020E4300701F43548FA30E709C3EA94F043
:1007BE0040150207DBC3EA940F50030207DB78FFF4
:1007CE0079FF7A0F0207DB780079007AF0C3E5240F
:1007DE009561500AC374019524500B0207F9E54A3E
:1007EE0020E70E0207F9E54A30E706884689478A70
:1007FE00482278A5E6FAC3E54933F8E54A33F912FB
:10080E0006BAE930E70BC3E89480E994FF40130180
:10081E0034C3E8947FE9940050020134787F790064
:10082E000134788079FFE820E715C3E52398F84076
:10083E0009C3E89401400302085B780102085BE8F3
:10084E00F424012523F8400302085B78FF884B222D
:10085E0078A6E6FAA847A9481206BAE930E70CC30B
:0F086E00E89401E994FF4016020890C3E894FF54
:10087D00E99400500302089078FF790002089078FF
:10088D000179FFE920E715C3E54B98F84009C3E866
:10089D00940140030208B778010208B7E8F4240177
:1008AD00254BF840030208B778FF88242278FF20F3
:1008BD00692879A1E76023E541601F74FF8541F048
:1008CD00848539F0306A0375F005A4F8C5F060022F
:1008DD0078FFC3E895645002A864886322C3E5409D
:1008ED0094C8E5419400E56350031401FB046002D4
:1008FD00F563220209032275E890227883E6FF3022
:10090D00EDF9A8BDA9BE0570C3E5709408405275F8
:10091D007000E9FA79A0E76044EA7007E571601BA1
:10092D0002093CC3E895716010E5715006600C1426
:10093D000209480460F9020948E571F571C3947222
:10094D00401B7561C0C394044013756180C394044A
:10095D00400B756140C39404400375610075BB097C
:10096D0022E5612410500274FFF5617982B704020B
:10097D002195C3A861E524985002A824C3E8956386
:10098D004002A86388258826E570B4070375BB105F
:10099D0022743279A787F0A4C5F0A2F733F8C3E823
:1009AD0095614002A861882288248825882688645C
:1009BD00227540007541F022C2AF75C820A8CCA9A0
:1009CD00CDAA3A30CF010A75C824D2AFC3EA13FAC3
:1009DD00E913F9E813F8AB3BAC3C883B893CC3E821
:1009ED009BF8E99C20690A547FF930660241E44185
:1009FD003EAD3D8A3DF9EA9D547FFA600678FF7958
:100A0D00FF4123AE3EAF3F8B3E8C3FA83BA93CC37D
:100A1D00E89EF8E99FF9C3E54113FBE54013FAE8B9
:100A2D002AF540E93BF54150067540FF7541FF4100
:100A3D008BAA40AB41AC40AD417E047F02C3EB9429
:100A4D0004400D1E1FC3EB94084005206A021E1FB3
:100A5D00C3ED13FDEC13FCDEF7C3EA9CFAEB9DFB33
:100A6D00EF6009C3E913F9E813F8DFF7EA28FAEBA9
:100A7D0039FB8A408B4150067BFF8B408B41C3EB8A
:100A8D0094025002D2663069047F0341B67892E633
:100A9D00FFC3E537948240110FC3E53794A04001A1
:100AAD000FC3EF940640027F057E02E541C4540F4B
:100ABD00F9E541C454F0F8E540C4540F28F8C3E8F3
:100ACD009EFAE99400FB4009C3EA9402EB940050AE
:100ADD00047A02E4FB6130AA40AB41EBC4FEEAC4E8
:100AED00540F4EFCC3EA9CFAEB9400FBC3E813C30E
:100AFD0013F8EA28FAEB3400FB8A408B41C3EB94E0
:100B0D00024002C2667802EBC4FE7B00EAC4540FB9
:100B1D004EFAC3EA98FA4005C3940250027A02785D
:100B2D0092E6FF3060026130855192855293D2601A
:100B3D0043E680C3E49AF8E49BF9C3E833F8E9335C
:100B4D00F930660261C3E8FAE9FBD3E913FDE81356
:100B5D00FC88518952C3EF94036038EF20E00DE813
:100B6D002CF8E93DF9ECFAEDFB020B8CE828F8E9DD
:100B7D0039F9C3E82402F8E93400F97AFE7BFFC3A2
:100B8D00EF9403400E8A538B54884D894E8C4F8DB4
:100B9D005061F7885389548A4D8B4E8C4F8D503050
:100BAD0069127553F07554FF754FF07550FF7551FF
:100BBD00F07552FF61F7E8FAD3E813FC8851C3EFE3
:100BCD0094036020EF20E007E82CF8ECFA61E3E8ED
:100BDD00282402F87AFEC3EF940340088A53884D07
:100BED008C4F61F788538A4D8C4FE568C3335002A3
:100BFD00646BF5683060028101753402D26043E6A2
:100C0D0080E52D5406602DA840A941C3E913F9E8EC
:100C1D0013F8306904E92440F9C2AF53E67F7591AA
:100C2D0000C3E498F594E499F595759104D2604369
:100C3D00E680D2AF22D264754300752000306C037C
:100C4D00752040020C61D264754300752040306CF4
:100C5D000375200078017901206620E52D5406608A
:0E0C6D0002C2647914E541C313700104F8C398
:100C7B00941440027814306904781B791BC3E83351
:100C8B00F8C3E933F9206010E543600C306903D5F4
:100C9B003404D26DA11791090543E59B5440B5204F
:100CAB0002A10130690908C3E8994001188190201D
:100CBB00640A08C3E899400281618190C264C2AFA3
:100CCB0053E67F7591003066127594007595F0753B
:100CDB009104D26043E680D2AF8161E5417EFFC3D0
:100CEB00334009C3334005C3334001FEC3E49E7553
:100CFB009400F59581DAC3E533940150028161309C
:100D0B0064028161D802A1158190C26DC2AF53E616
:100D1B007F759100855394855495759104854D92FB
:100D2B00854E93D26043E680D2AFE52D5406600822
:100D3B00206A020533020D53306D0D206C0A2064BE
:100D4B000715811581021641227800306402780163
:100D5B00E53775F007A4F9E5F028F5F0E9A2F013F3
:100D6B00A2F113A2F213F537C394785003753778B9
:100D7B00C3E53795384008D265C292C294C296300B
:100D8B006002A18A854F92855093D26043E6802200
:100D9B00D287207D16C2AF754202C295D2933062C4
:100DAB0002D296D2AF759F80020F97C2AF754202E7
:100DBB00C295D297306202D292D2AF759F80020F4A
:100DCB0097C287307243207D20C2AF7542039001DA
:100DDB0065757B20C296C297306204D294A1ECD287
:100DEB0095D2AF759F89020F97C2AF7542039001E1
:100DFB0065757B20C292C293306204D294C10CD22F
:100E0B0095D2AF759F81020F97207D17C2AF7542A8
:100E1B0003900140C296306202D294D2AF759F8983
:100E2B00020F97C2AF754203900140C2923062022B
:100E3B00D294D2AF759F81020F97D287207D16C2B5
:100E4B00AF754204C293D297306202D294D2AF757F
:100E5B009F81020F97C2AF754204C297D293306243
:100E6B0002D294D2AF759F89020F97C2873072431B
:100E7B00207D20C2AF754205900154757B08C2944A
:100E8B00C295306204D292C196D293D2AF759F8035
:100E9B00020F97C2AF754205900176757B80C294A5
:100EAB00C295306204D296C1B6D297D2AF759F80ED
:100EBB00020F97207D17C2AF754205900136C29481
:100ECB00306202D292D2AF759F80020F97C2AF757C
:100EDB00420590014AC2943062EBD296D2AF759F15
:100EEB0080020F97D287207D16C2AF754206C2973C
:100EFB00D295306202D292D2AF759F89020F97C200
:100F0B00AF754206C293D295306202D296D2AF75BC
:100F1B009F81020F97C287307244207D20C2AF752C
:100F2B004201900176757B80C292C293306204D2EB
:100F3B0096E140D297D2AF759F81020F97C2AF75E2
:100F4B004201900154757B08C296C297306205D25C
:100F5B0092020F61D293D2AF759F89020F97207DBA
:100F6B0017C2AF75420190014AC292306202D2960B
:100F7B00D2AF759F81020F97C2AF754201900136B8
:100F8B00C296306202D292D2AF759F89C26522900F
:100F9B000134757B00C292C294C296C293C295C2B1
:100FAB0097C262227880760908760908760408765B
:100FBB00FF0876030876FF087609087603087601A2
:100FCB00087601788C76010876FF0876FF0876FFA5
:100FDB000876FF0876FF0876030876FF0876FF0889
:100FEB0076FF0876250876D008762808765008769E
:100FFB00040876FF08760208760008767A0876FFF2
:10100B000876010876010876000876030876002238
:10101B007887E6FFC272BF0302D2727888E6C39468
:10102B00036008C27DE630E102D27DC27E7889E69C
:10103B0030E102D27EC3EF94026008758E01D27349
:10104B00021053758E00C273227880E614900080D4
:10105B009378A5F67881E6149000809378A6F678BD
:0F106B0086E61490008D9378A7F67886E6F5391F
:10107A00C394025003753902789CE67538FFB402AE
:10108A00037538A0B4030375388278A3E614900078
:10109A009A93F566120F9A22C2A4C2A0789DE6B46A
:1010AA000104D2A4C2A0B40204C2A4D2A022789697
:1010BA00E6FA7897E6FB7888E6B40305C3EB940E64
:1010CA00FB307F047A007BFFC3EB9AFCC394825007
:1010DA00027C827572000572EC8572F0A4C3E5F099
:1010EA00947D40F222D27F11B81206011206017ACB
:1010FA00007B007C101205F7E55C2AFA74003BFBC2
:10110A00DCF37C04C3EB13FBEA13FADCF7FEC27FC1
:10111A0011B822757C00757D00E5EF20E603752085
:10112A00000520903FFFE520146006901FFF146021
:10113A00009304600375EF1653D9BF7581C043FF4E
:10114A00801205F275EF0643B203E5B3240220E7E5
:10115A000DF521E5E320E0068521B343E301120FF3
:10116A009A7580FF75A48075F1F075D4BF759002E9
:10117A0075A5FC75F2FD75D50275A61175A0EE75FB
:10118A00F3F175E241120F9AE4F8F6D8FD75680199
:10119A00120FAF12169A78988673753001C2AF1281
:1011AA00060B12061B12060112062212060112066D
:1011BA0029120601C2AF757C00757D0078FA79FAAA
:1011CA00308607D9FBD8F7021C00111B115411A253
:1011DA0011B878988673120F9A75A90075B680753A
:1011EA007A0075881075890275C82475910475D8B6
:1011FA004075A82275B80275E690759B80759D00AA
:10120A0075D10E75BCC075BB0975BA1175E8801227
:10121A0005F2D2AF12090075360053DACF207E03E9
:10122A0043DA20307E0343DA1043DA01C2D8C271AE
:10123A0012060BD2617B037A0CE55B70077A0CDB32
:10124A00030211BE1206012070030211BEC270E52C
:10125A005CC3940240E1E52F541F855E5DF55EB5DF
:10126A005DD5DAD5C26153DACF207E0343DA203066
:10127A007E0343DA10C2D8C27178A2E67008D2742B
:10128A00E52F54E0F52FC275752900120606307451
:10129A0009C3E529940A4002D2751205F77802308B
:1012AA0074027800C3E55C9840F0C2AF12061B12C4
:1012BA00061B12061BD2AF12060B754C007888E685
:1012CA00B4030261BA1205F7788CE6C3940150039D
:1012DA000213BAE530C3940150030213BA757CA510
:1012EA00757DF1207435C3E55C94FF50030213BA8F
:1012FA00C2AF120630D2AF120606C3E55C940150A3
:10130A00EFC2AF12061B1205FC12061BD2AF120661
:10131A0006C3E55C94FF40E90218527F02D27F11AE
:10132A00B8120606C2AFC27F11B8AE5CC3E55C94C0
:10133A007FD2AF500261CA1205F2C2AF120630D292
:10134A00AFDFDA11EFC3EE7897F612060B1217D554
:10135A007F0AD27F11B8120606C2AFC27F11B8AE99
:10136A005CC3E55C947FD2AF50E61205F2C2AF12BD
:10137A00061B1205FC12061BD2AFDFD611EFEE24B4
:10138A00037896F6F87997E7C39482400398500653
:10139A00E824827897F612060B1216E8121804123D
:1013AA00060611B8C3E55C94FF500241E7021852E1
:1013BA00757C00757D00C3E55C954C4003855C4CEB
:1013CA0012060678017988E7B403027805C3E55C5A
:1013DA0098400241C7C2AF120630120630120630D8
:1013EA00D2AF12060B753000E4F531F5320531E55E
:1013FA0031F4703F0532789AE6781914601278321F
:10140A0014600D787D14600878FA14600375320050
:10141A00C3E53298401D120F9A1205F21532753142
:10142A000078998673C2AF120630D2AF7898867365
:10143A001206061205FCE52A700530740221BE78F0
:10144A00012074027806C3E55C9840A17888E6C357
:10145A0094036003120606E52A70030211BEC2AFA6
:0E146A00120F9AE4F522F523F524F525F52658
:10147800F567D2AF7885E6C333F565E4F544F545FD
:10148800F546F547F548F570F52CF52DF5377570E7
:101498000875BB101205F212090430EDFDA8BDA9AC
:1014A800BEE97001F8887112090875700875BB10DB
:1014B800111BC2AF7561FF12099E852261852262E8
:1014C800852263D2AF752201752401752501752621
:1014D80001856069756A0175B69075A903757A0109
:1014E8007888E6B40307C27D307602D27DD268D20E
:1014F80069753300120EEF120F201209BE1209C5CA
:101508001209BE1209C51209BE120C531207111294
:101518000D54120D9B1209C5120C42306E031207AE
:101528006D2066031208BA3066031208EA120D54D9
:10153800120DCC1209C5120C53306E031207A212F9
:101548000D54120E451209C5120C42306E031208D2
:1015580000120D54120E761209C5120C53306E0388
:1015680012085E120D54120EEF1209C51209041268
:101578000C42120D54120F201209081209C53069C5
:1015880032856461856462856069756A0179187A53
:101598000CC3E53399400FC269D26A8A3585646104
:1015A8008564630215BBC3E55C9401400302151111
:1015B800021649306A25206C22E535147006C26A85
:1015C800D26BA111F535C3E55C94014003021511F6
:1015D8007888E6C39403600302164975360078FAE2
:1015E80079A4E760027803C3E55F98505430740427
:1015F800E52A604D7888E6B40317207D0520760734
:10160800C119307602C119206C07D26C856461A1BA
:101618005078F0306C058564617820C3E5419850B6
:1016280002A111306C1BC26CC27D307602D27DD211
:101638006A753512856461A1110536E55C6002C1E1
:101648004C753600C2AF120F9A7887E6FE76021103
:101658001B7887EEF6E4F522F523F524F525F52623
:10166800F565752C00752D0075A90075B680757A1D
:1016780000D2AF120606120F9A78A4E66006D2923C
:10168800D294D296307409C3E5369404400221BE40
:1016980061F2901A0D782012172AE520B4550CA390
:1016A80012172AE520B4AA030216C8757CA5757D11
:1016B800F1120FAF1216E8757C00757D000216E76F
:1016C800901A0378807B0A12172AA308DBF9901A6C
:1016D8000F788C7B1912172AA308DBF9901A282295
:1016E800C2AF12176D12174A901A00740E12172FF4
:1016F800A3740912172FA3741512172F901A0378C1
:10170800807B0A12172EA308DBF9901A0F788C7BBE
:101718001912172EA308DBF912178012175E901AF8
:101728002822E493F622E6438F01538FFDFFC3E599
:1017380083941C400122EF857CB7857DB7F0538FD9
:10174800FE22438F02438F01857CB7857DB7901AAF
:101758000DF0538FFC22901A0D7455F12F901A0E2C
:1017680074AAF12F227A3079D07820901A40F12A81
:10177800E520F709A3DAF7227A3079D0901A40E702
:10178800F12F09A3DAF922AB74A875BB010279809D
:10179800BB02027981BB03027982BB04027984BB54
:1017A80005027986BB06027992BB07027987BB08D6
:1017B8000279A3BB0902799CBB0A027988BB0B0298
:1017C8007989E8F7227C0512060BDCFB22C2AF12EE
:1017D800061B1206221206291206301205FC1206F2
:1017E8001B1206221206291206301205FC12061BCD
:1017F800120622120629120630D2AF22C2AF1206F2
:101808003012062912062212061B1205FC12063097
:1018180012062912062212061B1205FC12063012A5
:10182800062912062212061BD2AF22AE74AF75C269
:10183800AF12061B12061B12061B1205FCDEF21263
:1018480006301205FCDFF8D2AF221217D51217CDD9
:101858001217CD75740175750175760011337C0505
:0E186800AD5C12060BC3ED955C70F5C3E55C3C
:101876009401400AC3E55C94FF403702189512179D
:101886008F1216E81217D5C2AF75EF161217CDDCF8
:10189600D10576C3E5769403500280C21217CD05B2
:1018A60075E5741490009F93F808C3E57598500287
:1018B60080A91217CD1217CD0574C3E574940C5088
:1018C600028095120FAF1216E8C2AF75EF16121707
:0118D600CD44
:0319FD0002111DB7
:101A00000E0915090904FF03FF0903010155AA0185
:101A1000FFFFFFFFFF03FFFFFF25D0285004FF0259
:091A2000007AFF0101000300FF40
:101A400023506C6174696E756D3530417633232097
:101A500023424C48454C492346333930232020202B
:101A60002020202020202020202020202020202076
:101C0000C2AFC2D353D9BF7581C043B20343FF8073
:101C1000752438752503B1DC7529A5752AF175E29F
:101C20004043F14053A4BF75D4FFD2867DFA7803B8
:101C300079E67C10752200752300901DE97B0675FE
:101C400024987525013086028145208608D8FBD965
:101C5000F9DCF781B7308608D8FBD9F9DCF781B712
:101C6000B19CE493A3C39A6004DDC381B7DBDBB10D
:101C70008E6002812E7B08E493FAA3B16FDBF87AC1
:101C800030B16F752200752300B18EEAFCEBFDC305
:101C9000ED94FE400EB18E8A278B28ED30E0048A49
:101CA000828B83B18E7AC270D8C3ED94FE601950D6
:101CB000CEBD002BEC600F7520007521FF7529004B
:101CC000752A000200008100A827A9280809D80465
:101CD000D90281DCB192EA89AAF281CE0D81A3C337
:101CE000ED94035053EDA2E092007AC5C3E58294CF
:101CF00000E583941C508A200010438F02438F011B
:101D00008529B7852AB7F0300029A827A92808090E
:101D1000438F01538FFDD804D902A133C3E58394C7
:101D20001C4003A3A11689AAE28529B7852AB7F02A
:101D3000A3A116538FFC817F7AC1BD030CE493A34A
:101D4000FAB153DCF8B14B817F8181AA22AB23B178
:101D50006FEBFAEA6222752608C3E52313F523E543
:101D60002213F52250066323A0632201D526EAB18F
:101D7000DCB1DC75260AEAF4200102D286300102C9
:101D8000C286B1DCC3134002C201D526EB22B19258
:101D9000EAFB208602A192308602A197752608AE42
:101DA00024AF25C3EF13FFEE13FEB1E0B1DCC3EAAD
:101DB000133086024480FA30E703632201C3E5232F
:101DC00013F523E52213F52250066323A0632201B5
:101DD000D526D9E52265236523F52222AE24AF2539
:101DE0000E0FDEFEDFFCD20122424C48656C6934E6
:071DF000373164F390060196
:00000001FF
